:100000000C946E000C9489000C948E0C0C94D60009
:100010000C9489000C9489000C9489000C9489003C
:100020000C9489000C9489000C948C070C9457084C
:100030000C948F080C9489000C9489000C9489000E
:100040000C9489000C9489000C9489000C9489000C
:100050000C948900721276126A125E126E12661287
:100060005A1256126212EE137A127E1282124F1236
:100070005F1371131E13E61232130C13D112BE124A
:10008000F91283139813AB13C613AC120672652CC6
:100090000375223B59781EBAE07A633BF47C75FF06
:1000A0004E7E3172117F0000000005813504F4831B
:1000B0002000018362463283200000816246307F47
:1000C0000000000582778C4F81432CE28217BF2409
:1000D00083A48DD981E1D8A180DB678211241FBE62
:1000E000CFE5D4E0DEBFCDBF10E0A0E6B0E0E4E4B1
:1000F000F7E302C005900D92AE3CB107D9F712E0CC
:10010000AEECB0E001C01D92A639B107E1F70C9446
:10011000B0040C94000081B3886281BB82B3877DF8
:1001200082BB84B3836084BB85B38C7F85BB87B37C
:100130008F6087BB88B3807F88BB08950F931F9320
:100140008C01C801AA2797FDA095BA2FBC01CD014B
:100150000E94F41817FF06C020E030E040E857E4A2
:100160000E94B61720E030E04AE755E40E948C195F
:10017000DC01CB01BC01CD010E94D718DC01CB0111
:100180000197F1F71F910F9108959B01AC01211583
:1001900031054105510549F080EA9FE00197F1F7EB
:1001A0002150304040405040F2CF08951F920F92AE
:1001B0000FB60F921124EF92FF920F931F932F937C
:1001C0003F934F935F936F937F938F939F93AF93DF
:1001D000BF93EF93FF938091280290912902A09101
:1001E0002A02B0912B028093730290937402A09321
:1001F0007502B0937602809193028823B1F1109238
:1002000093028091CA0199278130910511F00297DC
:1002100061F59798969880912E028E7F80932E029A
:1002200080912E0299279F938F9384E0F82EFF925E
:1002300000E610E01F930F930E94D50980912E02D3
:100240008D7F80932E0280912E0299279F938F930A
:10025000FF921F930F930E94D5098DB79EB70A9600
:100260000FB6F8949EBF0FBE8DBF0E941A0B8091EF
:10027000040290910502A0910602B0910702009736
:10028000A105B105A1F08091040290910502A09111
:100290000602B09107020197A109B10980930402F7
:1002A00090930502A0930602B093070285C0809147
:1002B0007F0290918002A0918102B0918202BC01E4
:1002C000CD010E94D718DC01CB01809304029093EA
:1002D0000502A0930602B093070280913402909128
:1002E0003502A0913602B091370220E030E048ECB0
:1002F00052E4BC01CD010E948C197B018C018091DC
:100300007F0290918002A0918102B09182029C01B3
:10031000AD01C801B7010E940018DC01CB01809338
:10032000280290932902A0932A02B0932B020E94E4
:10033000960A80916802992782309105B1F0833046
:1003400091051CF4019721F037C00397D9F034C010
:100350008091280290912902A0912A02B0912B024B
:1003600020E030E040E251E419C0809128029091F1
:100370002902A0912A02B0912B0220E030E040E750
:1003800052E40CC08091280290912902A0912A0287
:10039000B0912B0220E030E048EC52E4BC01CD01EA
:1003A0000E948C19DC01CB018093280290932902D2
:1003B000A0932A02B0932B0280912202882391F00D
:1003C000829B10C08091730290917402A09175027B
:1003D000B09176028093280290932902A0932A027A
:1003E000B0932B0280919202882331F08091920287
:1003F00081508093920201C0949880913C0288239E
:1004000021F080913C02815001C088EC80933C0235
:100410008091CA019927009721F0019709F4BEC085
:100420009BC1E0902802F090290200912A021091CD
:100430002B0280918D0290918E02A0918F02B0913B
:1004400090029C01AD01C801B7010E941B1918164A
:1004500094F480918D0290918E02A0918F02B091C0
:10046000900220E030E040E050E0BC01CD010E946D
:100470001B1987FF2AC0E0902802F0902902009102
:100480002A0210912B0280918D0290918E02A091F0
:100490008F02B09190029C01AD01C801B7010E948A
:1004A00018198823BCF480918D0290918E02A0913E
:1004B0008F02B091900220E030E040E050E0BC01BB
:1004C000CD010E94181988232CF4979A80912E024E
:1004D000816004C0979880912E028E7F80932E02B7
:1004E00080912E0299279F938F9384E08F9380E6CB
:1004F00090E09F938F930E94D5090F900F900F90DB
:100500000F900F90E0902802F090290200912A02AB
:1005100010912B0280916A0290916B02A0916C0263
:10052000B0916D029C01AD01C801B7010E941B1979
:10053000181694F480916A0290916B02A0916C025B
:10054000B0916D0220E030E040E050E0BC01CD0110
:100550000E941B1987FFE3C0E0902802F090290257
:1005600000912A0210912B0280916A0290916B02F5
:10057000A0916C02B0916D029C01AD01C801B70160
:100580000E94181988230CF0CFC080916A029091C4
:100590006B02A0916C02B0916D02B7C0E0908D0229
:1005A000F0908E0200918F021091900280916A0269
:1005B00090916B02A0916C02B0916D029C01AD0113
:1005C000C801B7010E94B517DC01CB01E0902802F9
:1005D000F090290200912A0210912B029C01AD019A
:1005E000C801B7010E941B1918166CF5E0908D0226
:1005F000F0908E0200918F021091900280916A0219
:1006000090916B02A0916C02B0916D029C01AD01C2
:10061000C801B7010E94B617DC01CB01E0902802A7
:10062000F090290200912A0210912B029C01AD0149
:10063000C801B7010E94181988232CF4979A809159
:100640002E02816004C0979880912E028E7F809345
:100650002E0280912E0299279F938F9384E08F938F
:1006600080E690E09F938F930E94D5090F900F90A2
:100670000F900F900F90E0902802F09029020091C7
:100680002A0210912B0280918D0290918E02A091EE
:100690008F02B09190029C01AD01C801B7010E9488
:1006A0001B19181694F480918D0290918E02A091DE
:1006B0008F02B091900220E030E040E050E0BC01B9
:1006C000CD010E941B1987FF2AC0E0902802F090FC
:1006D000290200912A0210912B0280918D029091A3
:1006E0008E02A0918F02B09190029C01AD01C801D1
:1006F000B7010E9418198823BCF480918D02909153
:100700008E02A0918F02B091900220E030E040E094
:1007100050E0BC01CD010E94181988232CF4969A50
:1007200080912E02826004C0969880912E028D7F67
:1007300080932E0280912E0299279F938F9384E0BD
:100740008F9380E690E09F938F930E94D5090F903E
:100750000F900F900F900F9078940E944D0A9091F7
:100760007A0280918702981750F080917A02992737
:1007700020918702821B9109039764F414C0809131
:100780007A02992720918702821B9109805C9F4FF2
:1007900003974CF060E18EEC90E00E9425098EEC0E
:1007A00090E00E94F013FF91EF91BF91AF919F9164
:1007B0008F917F916F915F914F913F912F911F91F9
:1007C0000F91FF90EF900F900FBE0F901F90189514
:1007D000F89444E050E06AE670E08FE692E00E9410
:1007E000E31544E050E06EE670E080E092E00E94A5
:1007F000E31541E050E064E670E08AEC91E00E948D
:10080000E31541E050E065E670E083E492E00E9489
:10081000E31541E050E06FE770E082E292E00E9471
:10082000E31544E050E06AE770E08BE092E00E945C
:10083000E31544E050E066E770E08DE892E00E9446
:10084000E31544E050E062E770E08AE692E00E943F
:10085000E31541E050E06EE770E089E792E00E9426
:10086000E31541E050E062E870E08CE892E00E941D
:10087000E31541E050E063E870E089EC91E00E940C
:10088000E31541E050E064E870E08DE392E00E94FF
:10089000E31544E050E066E670E08FE792E00E94E6
:1008A000E31541E050E065E870E088E692E00E94E0
:1008B000E3157894089510926F02109270021092CE
:1008C0007102109272028AE097EDA3E2BCE380937A
:1008D000000290930102A0930202B093030220E071
:1008E00030E048EC52E420937F0230938002409342
:1008F00081025093820261E06093CA0182E080939A
:1009000043021092220284EF91E0A0E0B0E08093D5
:100910000B0290930C02A0930D02B0930E0280E0A4
:1009200090E0AAEFB3E480938D0290938E02A0939F
:100930008F02B093900220936A0230936B0240932F
:100940006C0250936D021092790260938C021092A7
:10095000C90160933D02109268020E94E803089565
:10096000CFE5D4E0DEBFCDBF789488E190E02FE002
:100970000FB6F894A89581BD0FBE21BDF89483E60B
:1009800090E00E94BF158F3F39F40E945B0460E045
:1009900083E690E00E94D8151092210244E050E0D6
:1009A0006AE670E08FE692E00E94C71580916F02C0
:1009B00090917002A0917102B09172028156994794
:1009C000AE4FBF4F8F5D984CA041B04058F0109291
:1009D0006F021092700210927102109272028AE6F7
:1009E0008093210244E050E06EE670E080E092E007
:1009F0000E94C715E0900002F090010200910202EF
:100A00001091030223EF3FEF47EC52E4C801B70116
:100A10000E941B19181654F027E137EB41ED58E3FB
:100A2000C801B7010E94181988237CF48AE097ED69
:100A3000A3E2BCE38093000290930102A093020220
:100A4000B09303028EE68093210244E050E066E614
:100A500070E08FE792E00E94C71580917F0290912D
:100A60008002A0918102B091820220EF33E244E73C
:100A700059E4BC01CD010E941B19181694F0809115
:100A80007F0290918002A0918102B091820220E0C9
:100A900030E040E85FE3BC01CD010E9418198823D3
:100AA0007CF480E090E0A8ECB2E480937F02909325
:100AB0008002A0938102B093820286E68093210295
:100AC00041E050E064E670E08AEC91E00E94C715D6
:100AD0008091CA01823030F081E08093CA0184E6BF
:100AE0008093210241E050E065E670E083E492E00B
:100AF0000E94C71580914302833030F082E08093DA
:100B0000430285E68093210241E050E06FE770E008
:100B100082E292E00E94C71580912202823028F082
:100B2000109222028FE78093210244E050E06AE7AE
:100B300070E08BE092E00E94C71580910B029091CB
:100B40000C02A0910D02B0910E0280549244AF406D
:100B5000B04078F084EF91E0A0E0B0E080930B0229
:100B600090930C02A0930D02B0930E028AE780933B
:100B7000210244E050E066E770E08DE892E00E94D8
:100B8000C71580918D0290918E02A0918F02B09135
:100B9000900220EF33E244E759E4BC01CD010E940A
:100BA0001B19181694F080918D0290918E02A091DD
:100BB0008F02B091900220E83FE443EC57ECBC0177
:100BC000CD010E94181988237CF480E090E0AAEF00
:100BD000B3E480938D0290938E02A0938F02B09322
:100BE000900286E78093210244E050E062E770E0E3
:100BF0008AE692E00E94C71580916A0290916B028A
:100C0000A0916C02B0916D0220EF33E244E759E409
:100C1000BC01CD010E941B19181694F080916A0244
:100C200090916B02A0916C02B0916D0220E83FE4BC
:100C300043EC57ECBC01CD010E94181988237CF4C9
:100C400080E090E0A8ECB2E480936A0290936B029B
:100C5000A0936C02B0936D0282E78093210241E081
:100C600050E06EE770E089E792E00E94C71580913E
:100C70007902853028F0109279028EE78093210264
:100C800041E050E062E870E08CE892E00E94C71515
:100C900080918C02823030F081E080938C0282E877
:100CA0008093210241E050E063E870E089EC91E03C
:100CB0000E94C7158091C901823028F01092C901A5
:100CC00083E88093210241E050E064E870E08DE326
:100CD00092E00E94C71580913D02823030F081E0A1
:100CE00080933D0284E88093210241E050E065E872
:100CF00070E088E692E00E94C71580916802843017
:100D000028F01092680285E88093210280912102E8
:100D1000882309F450C088E10FB681BD11BC0FBE15
:100D20000E94E803789481E00E94600708E412E0E2
:100D300085E492E5A2E5B0E08093480290934902F1
:100D4000A0934A02B0934B02809121024AE050E006
:100D500060ED71E099270E94F815BC01C8010E945E
:100D60005C161F921F930F930E94D5090E944D0A93
:100D700068EE73E080E090E00E94C5000E944D0A9A
:100D800068EE73E080E090E00E94C5000E944D0A8A
:100D900068EE73E080E090E00E94C500A89588E1CD
:100DA00090E02FE00FB6F894A89581BD0FBE21BD4D
:100DB0000F900F900F9085B58F6085BD89B78068C3
:100DC00089BF8DE983BD0E948B000E94B20C81B364
:100DD000806C81BB8C9A10928302109284021092D4
:100DE000850210928602109204021092050210925F
:100DF0000602109207021092CC011092CD011092BF
:100E0000CE011092CF010E94B40A789481E00E9432
:100E100060071F9281E690E09F938F930E94D5090F
:100E200064EF71E080E090E00E94C50086E595E403
:100E3000A2E5B0E08093480290934902A0934A0251
:100E4000B0934B0282E090E09F938F9381E08F9369
:100E50004AE050E060ED71E088EF90E00E94F81504
:100E6000BC0188E492E00E945C169F938F930E94DD
:100E7000D50968EE73E080E090E00E94C5008DB770
:100E80009EB708960FB6F8949EBF0FBE8DBF809197
:100E90003D02882391F00E9439081F9288E690E075
:100EA0009F938F930E94D50968EE73E080E090E0F5
:100EB0000E94C5000F900F900F900E94EB10FDCF85
:100EC000982F10921F0110921E0110924101109252
:100ED0004001813051F4BE9887B3806B87BB1DB849
:100EE0008DB1816D8DB9C49A0AC0882341F4BE9A30
:100EF00087B38F7487BB9DB98DB1806C8DB98EB16E
:100F00008FB181E080931F020895F89410921F0121
:100F100010921E01789408951F920F920FB60F92AF
:100F200011242F933F934F935F936F937F938F93EE
:100F30009F93AF93BF93EF93FF936C9B03C0C49AAF
:100F40000000C49880911E018F5F8F7380934201CF
:100F50008091420180931E019091420180911F0176
:100F6000981729F40E94850781E080931E018091E3
:100F70001E01E82FFF27E252FF4F8FB1808390912F
:100F8000400180914101981799F0809141018F5F54
:100F90008F7180934301809143018093410180913F
:100FA0004101E82FFF27E05EFE4F80818FB905C029
:100FB00081E080931F026C99C49AFF91EF91BF91D9
:100FC000AF919F918F917F916F915F914F913F91E1
:100FD0002F910F900FBE0F901F90189590911E01AA
:100FE00080911F019817D1F380911F018F5F8F733C
:100FF00080931F01E82FFF27E252FF4F808199273E
:101000000895FC0180911F028823E1F36C99C49834
:101010006F9810921F0280818FB991E09617E0F4CB
:10102000DF011196962F91503D91209140012F5F45
:101030002F7180914101281729F46F9A8091410105
:101040002817E1F3E22FFF27E05EFE4F3083209365
:101050004001915049F7962F6F9A892F992708954B
:10106000F8941092410110924001789408950895E7
:10107000089580E189B988E98AB986E880BD80E071
:101080008093870280937A0280932D028093F001EF
:1010900080936E0208958AB187708AB908958FB7D8
:1010A000F89410927A02109287028FBF08951F92CF
:1010B0000F920FB60F9211242F933F934F935F938C
:1010C0006F937F938F939F93AF93BF93EF93FF9310
:1010D0009CB190934401E0917A02EF5FEF73E0934B
:1010E0004501E0937A0280918702E81719F40E9483
:1010F0004F0804C0FF27E85BFE4F9083FF91EF91FC
:10110000BF91AF919F918F917F916F915F914F911F
:101110003F912F910F900FBE0F901F9018951F9227
:101120000F920FB60F9211248F939F93EF93FF931B
:101130009091F00180912D02981789F080912D02F5
:101140008F5F8F718093460180932D02E82FFF27D8
:10115000E857FE4F8081809347018CB901C05598B4
:10116000FF91EF919F918F910F900FBE0F901F9065
:10117000189590917A02809187029817D1F3809107
:1011800087028F5F8F7380938702E82FFF27E85BCA
:10119000FE4F808199270895282F9091F0019F5F3D
:1011A0009F7180912D029817E1F3E92FFF27E857EF
:1011B000FE4F20839093F001559A089520E030E08F
:1011C00090917A0280918702981711F021E030E027
:1011D000C901089520E030E09091F00180912D0246
:1011E000981711F021E030E0C90108958FB7F89405
:1011F0001092F00110922D028FBF089580E00E949E
:10120000CC088DE00E94CC088AE00E94CC080895AA
:10121000A0E0B0E0EEE0F9E00C94091B7C01DD24D5
:10122000CD2DDD278E010E0D1F1DF80180810E943E
:10123000CC08F8018081882311F0D394F1CFCE013E
:10124000E7E0CDB7DEB70C94251BCF92DF92FF927B
:101250000F931F93CF93DF93CDB7DEB721970FB6D0
:10126000F894DEBF0FBECDBF8C01F62E90E096172E
:10127000C8F4680199830E94B908F60180839981B6
:101280008D3021F08A3011F0882331F4F60110827C
:101290009F5F892F99270EC09F5F0894C11CD11CA6
:1012A0009F1540F3892F9927080F191F01501040EF
:1012B000F801108221960FB6F894DEBF0FBECDBFA5
:1012C000DF91CF911F910F91FF90DF90CF90089504
:1012D000BC0188E492E00E946E1688E492E00E94CD
:1012E00008090895982FE0917A02EF5FEF73E09379
:1012F0007A0280918702E81719F40E944F08089536
:10130000FF27E85BFE4F9083089508950F931F9386
:10131000CF93DF93EC0100E08881882361F0FE0128
:10132000E00FF11D80810E9472090F5FFE01E00F46
:10133000F11D8081F2CF1127C00FD11F88810E943B
:101340007209C801DF91CF911F910F9108950F93FA
:101350001F93CF93DF93262F8C013327211531055F
:1013600041F0E901F80181918F010E94CC08219799
:10137000C9F7DF91CF911F910F9108950F931F939C
:10138000CF93DF93262F8C0133272115310541F0B0
:10139000E9010E94B908F80181938F012197C9F7EB
:1013A000DF91CF911F910F910895A0E0B0E0EBED98
:1013B000F9E00C94051B0E851F8588899FB6F8946B
:1013C00051E1C52ED12CCC0EDD1E5601E82EFF2496
:1013D000E2FE06C089898093A8018093FA0140C08B
:1013E0008091A8018093FA01B80181EF91E00E94F9
:1013F0006716F80101900020E9F73197E01BF10B27
:1014000026E02E1BA1F0422F552790E235E0E5EFB4
:10141000F1E080818183315031973323D1F7FA0194
:10142000E21BF109EF50FE4F9083215079F71092A3
:10143000F701E0FE09C082E090E0C80ED91EF50178
:1014400080818093F80102C01092F801E1FE06C08D
:10145000F60180818F5F8093F90102C01092F9013B
:1014600020E0E1EFF1E039E08191082E82958025BE
:10147000082E8695869580259927019695958795BE
:1014800081709070280F315037FFEECF2068209385
:10149000FB019FBEEBE00C94211BA8956BE081EF54
:1014A00091E00E9401080E94EE07482F282F332761
:1014B000C9018095909564E0959587956A95E1F7C7
:1014C0008F7090702F70307028173907E9F44093AF
:1014D000200280912002282F33272F7030708091B6
:1014E000080299278F709070821793074CF4949993
:1014F00004C080918C028111949A85E080939202BD
:1015000080912002809308020E9485070895982FF9
:101510008FEF8ABBAD9AAA9A000000009BBB000027
:101520000000AA9800000000AA9A0895AE9A8FEFD2
:101530008ABBAD9AAA9A84E08BBBAA98AA9AAE9865
:1015400088E080932C02E0916E00F0916F00108291
:1015500081E0809393021092880210928902109287
:101560008A0210928B0208958B98939A8A98929A85
:1015700084B38C6F84BB1092440210924502109287
:1015800046021092470210922F02109230021092DF
:10159000310210923202AA9AAB9AAC98AE9AAF9AE4
:1015A000AE9880E20E94870A809143029927813099
:1015B000910559F0823091051CF4892B21F010C05F
:1015C000029741F00DC087E601C088E70E94870AB4
:1015D00080EC04C088E70E94870A83EC0E94870A97
:1015E000AE9A8FEF8ABBAD9AAA9A84E08BBBAA9879
:1015F000AA9AAE9888E080932C02E0916E00F09158
:101600006F00108281E08093930210928802109202
:10161000890210928A0210928B0208951ABAAD9A2A
:10162000AB9A00000000AB980000000089B3AB9AB1
:1016300099270895EF92FF920F931F930E940E0B2C
:10164000182F83E00E94870A1ABA1BBAAD9810922D
:101650004402109245021092460210924702AB9A41
:1016600000000000AB980000000089B3282F33274A
:10167000442755278091440290914502A09146024B
:10168000B0914702822B932BA42BB52B809344025D
:1016900090934502A0934602B0934702AB9A000094
:1016A0000000AB980000000089B39927AA27BB2748
:1016B0002227382F492F5A2F8091440290914502BA
:1016C000A0914602B0914702822B932BA42BB52BFD
:1016D0008093440290934502A0934602B093470240
:1016E000AB9A00000000AB980000000089B3992776
:1016F000AA27BB27AC01332722278091440290916F
:101700004502A0914602B0914702822B932BA42B55
:10171000B52B8093440290934502A0934602B09368
:101720004702AB9A10932C0213FF09C010922F02AC
:101730001092300210923102109232020CC08FEFE0
:101740009FEFAFEFB0E080932F0290933002A09311
:101750003102B093320280912F0290913002A09119
:101760003102B0913202582F44273327222780912B
:10177000440290914502A0914602B0914702822B0B
:10178000932BA42BB52B8093440290934502A093F6
:101790004602B09347028091440290914502A09185
:1017A0004602B0914702815C914EA44EB0406CF469
:1017B0008091440290914502A0914602B091470267
:1017C00080549E41AB41BF4F24F481E080930902D5
:1017D00002C01092090220914402309145024091CA
:1017E0004602509147028091880290918902A0910F
:1017F0008A02B0918B02281B390B4A0B5B0B57FFF7
:1018000007C050954095309521953F4F4F4F5F4F02
:10181000215A364841405040BCF080918802909156
:101820008902A0918A02B0918B0280934402909326
:101830004502A0934602B0934702949A85E08093B4
:10184000920281E0809309028091440290914502C6
:10185000A0914602B091470280938802909389023A
:10186000A0938A02B0938B0280914402909145022A
:10187000A0914602B0914702BC01CD010E94F4182C
:10188000DC01CB01E0900002F09001020091020225
:10189000109103029C01AD01C801B7010E948C198F
:1018A000DC01CB018093340290933502A093360281
:1018B000B0933702E0903402F09035020091360286
:1018C0001091370280917B0290917C02A0917D0261
:1018D000B0917E029C01AD01C801B7010E94B6170C
:1018E000DC01CB018093340290933502A093360241
:1018F000B09337021F910F91FF90EF900895982FAA
:101900008FEF8ABBAD98AA9A000000009BBB000035
:101910000000AA9800000000AA9A08951F920F9252
:101920000FB60F9211240F900FBE0F901F901895B5
:10193000EF92FF920F931F937B018C0181E00E9435
:10194000870A8E2D0E947F0C8F2D0E947F0C802F86
:101950000E947F0C88E00E94870A1F910F91FF90E0
:10196000EF90089514BA8FEF85BB81E08093FC015E
:101970008093FD018093FE018093FF01109242024B
:1019800080930A02109227020895EF92FF920F931C
:101990001F93CF93DF938091200280FD63C18091DC
:1019A00009028823C1F080913C028536A0F01F9285
:1019B00080E790E09F938F930E94D5090F900F903E
:1019C0000F90949904C080918C028111949A85E0C3
:1019D0008093920243C110917902812F992787FD4C
:1019E0009095A92FB92FBC01CD010E94F41817FFC3
:1019F00006C020E030E040E853E40E94B6179B01A7
:101A0000AC0160E070E080E291E40E94DA19DC0150
:101A1000CB01E0902802F090290200912A02109157
:101A20002B029C01AD01C801B7010E948C19DC0199
:101A3000CB0120E030E040E05FE3BC01CD010E943B
:101A4000B617DC01CB01BC01CD010E94FE18DC0100
:101A5000CB01BC01CD010E94D718DC01CB018093E2
:101A6000230290932402A0932502B09326022AE039
:101A700030E048E452E0BC01CD010E941D16809187
:101A80007902282F332708E412E0F80101900020A2
:101A9000E9F72E1B3F0B265B3D4F409123025091EF
:101AA0002402609125027091260277FF02C02F5F09
:101AB0003F4F1216130644F580E077FF04C08DE215
:101AC0008093D00181E040E0421750F4E82FFF27D7
:101AD00090E3E053FE4F422F91934150E9F7422F9C
:101AE0009927FC01E40FF11DE053FE4F1082885B43
:101AF0009D4FBC0180ED91E00E945C1660ED71E0AD
:101B000088E492E00E9467168091200283FF48C01B
:101B10008091CA018150823008F042C08091200239
:101B200080FDFCCF8091200283FDF8CF80912002C0
:101B300081FDF4CF8091200282FDF0CF1F9287E7D4
:101B400090E09F938F930E94D5090F900F900F9074
:101B50008091200280FD0CC08091200283FD08C08E
:101B60008091200281FD04C08091200282FFF0CF8D
:101B70008091200280FF04C0F8940E94960A789415
:101B80008091200280FDFCCF8091200283FDF8CF60
:101B90008091200281FDF4CF8091200282FDF0CF60
:101BA000C8E4D2E0F80101900020E9F73197EC1B7E
:101BB000FD0BE730F10508F441C08E2F8650082F49
:101BC0001127075B1D4FB80180E192E00E94671664
:101BD000F80110820FE012E08BE580930F028091F4
:101BE0002002992796958795969587959C01217057
:101BF000307080FF0DC0BE01C8010E9467161F92A1
:101C00001F930F930E94D5090F900F900F9026C03D
:101C10003F932F938091790299279F938F9383E02D
:101C20008F931F930F930E94D5098DB79EB7079688
:101C30000FB6F8949EBF0FBE8DBF10C08091790281
:101C400099279F938F9381E08F93DF93CF930E9487
:101C5000D5090F900F900F900F900F908091200258
:101C600080FF9DCEE6E0CDB7DEB70C94261BEF9249
:101C7000FF920F931F93CF93DF937B018C01EA01B7
:101C8000C801B7010E941D16FE0101900020E9F76E
:101C90003197EC1BE63040F536E03E1B1E8225E016
:101CA000632F7727AB01415050404530510574F404
:101CB000DE01A20FB11DFD01E61BF70B80818C93A5
:101CC0002150822F99274817590794F317FD3F5F3A
:101CD000332331F080E3FE01232F81932150E9F774
:101CE00017FF02C08DE28883CE01E6E0CDB7DEB7F4
:101CF0000C94261BA0E0B0E0E0E8FEE00C94061B8C
:101D00005C018050924079F4809100029091010230
:101D1000A0910202B091030220E030E543EC57E4C9
:101D2000BC01CD0127C010917902812F992787FD31
:101D30009095A92FB92FBC01CD010E94F41817FF6F
:101D400006C020E030E040E853E40E94B6179B0153
:101D5000AC0160E070E080E291E40E94DA19DC01FD
:101D6000CB01F501E080F180028113819C01AD017E
:101D7000C801B7010E948C19DC01CB0120E030E0E2
:101D800040E05FE3BC01CD010E94B617DC01CB014E
:101D9000BC01CD010E94FE18DC01CB01BC01CD01CC
:101DA0000E94D718DC01CB01809323029093240278
:101DB000A0932502B09326028091230290912402E1
:101DC000A0912502B09126022AE030E048E452E0DA
:101DD000BC01CD010E941D16C8E4D2E0FE010190B5
:101DE0000020E9F73197EC1BFD0B379798F01F9215
:101DF0008DE790E09F938F930E94D50968EE73E082
:101E000080E090E00E94C50080E090E00F900F908D
:101E10000F90E6C08091230290912402A0912502A8
:101E2000B09126022AE030E0AE01BC01CD010E9453
:101E3000370EC5E062C08091200280FD62C08091B3
:101E4000200281FF1AC0EC2FFF27E85BFD4F808145
:101E50008F5F8083CC2349F48E3211F480E380833A
:101E600080818A3331F48DE203C08A3311F480E338
:101E700080838091200281FDFCCF8091200282FF2F
:101E800009C0CC2311F4C5E001C0C15080912002EB
:101E900082FDFCCF28E432E08C2F9927F0E0AF16CA
:101EA000F2E0BF06A9F49F938F9385E090E09F93A3
:101EB0008F9383E08F933F932F930E94D5098DB723
:101EC0009EB707960FB6F8949EBF0FBE8DBF15C084
:101ED0009F938F938091790299279F938F9383E0AB
:101EE0008F933F932F930E94D509EDB7FEB7379696
:101EF0000FB6F894FEBF0FBEEDBF8091200283FFA6
:101F00009ACF8091200299279C012170307080FF28
:101F100066C028E432E0F0E0AF16F2E0BF0611F54B
:101F20004AE050E060E070E0C9010E948516DC01E3
:101F3000CB01BC01CD010E94F418DC01CB0120E0F3
:101F400030E543EC57E4BC01CD010E940018DC01F0
:101F5000CB018093000290930102A0930202B09300
:101F600003023AC04AE050E060E070E0C9010E941C
:101F70008516DC01CB01BC01CD010E94F4186B0178
:101F80007C0110917902812F992787FD9095A92FC7
:101F9000B92FBC01CD010E94F41817FF06C020E044
:101FA00030E040E853E40E94B6179B01AC0160E0CA
:101FB00070E080E291E40E94DA19DC01CB019C011F
:101FC000AD01C701B6010E940018DC01CB01F5018B
:101FD00080839183A283B38381E090E001C0C90133
:101FE000EAE0CDB7DEB70C94221B1F93CF93DF93AB
:101FF000EC012AE030E048E452E0688179818A818E
:102000009B810E941D16A8E4B2E0FD010190002012
:10201000E9F73197EA1BFB0B379798F01F928DE792
:1020200090E09F938F930E94D50968EE73E080E063
:1020300090E00E94C50080E090E00F900F900F901C
:1020400069C02AE030E0AD01688179818A819B8195
:102050000E94370E15E040C08091200280FD40C0F4
:102060008091200281FF1AC0E12FFF27E85BFD4F1E
:1020700080818F5F8083112349F48E3211F480E3D5
:10208000808380818A3331F48DE203C08A3311F476
:1020900080E380838091200281FDFCCF809120022B
:1020A00082FF09C0112311F415E001C01150809185
:1020B000200282FDFCCF812F99279F938F9382E08E
:1020C0008F9388E492E09F938F930E94D5090F909D
:1020D0000F900F900F900F908091200283FFBCCF44
:1020E0008091200299279C012170307080FF11C0DF
:1020F0004AE050E060E070E088E492E00E948516DB
:10210000DC01CB0188839983AA83BB8381E090E0C3
:1021100001C0C901DF91CF911F9108951F93CF9303
:10212000DF93EC01162F88814AE050E060ED71E00A
:1021300099270E94F815BC0188E492E00E94671676
:1021400032C08091200280FD32C08091200281FF48
:1021500011C040914802242F3327812F9927C09620
:10216000281739071CF44F5F4093480280912002E2
:1021700081FDFCCF8091200282FF0BC0809148023C
:10218000813318F08150809348028091200282FDB3
:10219000FCCF1F9288E492E09F938F930E94D50911
:1021A0000F900F900F908091200283FFCACF8091F3
:1021B000200299279C012170307080FF07C088E4BD
:1021C00092E00E949215888321E030E0C901DF91FE
:1021D000CF911F9108951F938091200280FDFCCF25
:1021E0008091200283FDF8CF8091200281FDF4CF01
:1021F0008091200282FDF0CF80910A02882309F0AD
:10220000C2C08091200280FD0CC08091200283FD1D
:1022100008C08091200281FD04C08091200282FFCD
:10222000F0CF6EE170E080E090E00E94C500809108
:10223000200280FD0CC08091200283FD08C08091A7
:10224000200281FD04C08091200282FFF0CF8091A6
:10225000200281FF18C080914202E82FFF27E4503E
:10226000FE4F8081823008F462C080914202882350
:1022700009F45DC080914202E82FFF27E450FE4F31
:102280008081815016C08091200282FF14C080910D
:102290002702882309F04BC080914202882309F469
:1022A00046C080914202E82FFF27E450FE4F808114
:1022B0008F5F80833CC08091200283FF1CC080918F
:1022C00042028823A1F180914202823031F41092BF
:1022D000420281E08093FC012AC080914202E82FF3
:1022E000FF27E450FE4F81E08083809142028150BD
:1022F000809342021CC08091200280FF11C0809117
:1023000042028330A0F4809142028F5F80934202A8
:1023100080914202E82FFF27E450FE4F81E0C9CFB1
:102320006EE170E080E090E00E94C50057C28091AD
:10233000200280FDFCCF8091200283FDF8CF8091A8
:10234000200281FDF4CF8091200282FDF0CF6EE16A
:1023500070E080E090E00E94C5008091200280FD46
:10236000FCCF8091200283FDF8CF8091200281FD77
:10237000F4CF8091200282FDF0CF6EE170E080E02A
:1023800090E00E94C50010920A02109227028091EC
:102390004202992781309105E9F0823091051CF4C1
:1023A000892B49F01BC28230910509F45FC0039765
:1023B00009F4B9C013C28091FC01813009F00EC24A
:1023C00011E0109327020E94C50C10930A0210938B
:1023D000420204C28091FD01813009F0FFC111E089
:1023E00010932702109223021092240210922502C9
:1023F0001092260280916F0290917002A09171025A
:10240000B09172020097A105B10551F183E292E00B
:102410000E94F50F8823F9F02091230230912402C5
:10242000409125025091260280916F029091700296
:10243000A0917102B0917202281739074A075B0711
:1024400079F02F523B4C4440504051F01093FC0126
:102450001092420202C08093420210930A02BEC14F
:1024600082E0809342021093FE01ADC18091FD0194
:1024700099278130910521F0029709F44EC0AEC131
:102480008091FE019927AA27BB27FC013197EE30E6
:10249000F10508F0A3C1E65DFF4F0C94351B81E008
:1024A000809327021F9283E890E02FC01F9288E854
:1024B00090E02BC01F928DE890E027C01F9280E92A
:1024C00090E023C01F9285E990E01FC01F928AE927
:1024D00090E01BC01F928FE990E017C01F9284EA22
:1024E00090E013C01F9289EA90E00FC01F928CEA1F
:1024F00090E00BC01F928FEA90E007C01F9284EB20
:1025000090E003C01F928AEB90E09F938F930E940C
:10251000D5090F900F900F9061C18091FE0181301D
:1025200009F05CC159C18091FD0199278130910565
:1025300021F0029709F44BC151C18091FE01992706
:10254000AA27BB27FC013197EE30F10508F046C100
:10255000E85CFF4F0C94351B81E0809327028FE6E7
:1025600092E00E94F50FF89444E050E06AE670E0D3
:102570008FE692E00E94E315789420C164E089E739
:1025800092E00E948E10882309F428C1F89441E05B
:1025900050E06EE770E089E792E00E94E3157894DE
:1025A0000DC162E083E492E00E948E10882309F45A
:1025B00005C1F8940E94B40A41E050E065E670E07D
:1025C00083E492E00E94E3157894F8C061E08AEC1D
:1025D00091E00E948E10882309F4F0C0F89441E045
:1025E00050E064E670E08AEC91E00E94E315789494
:1025F000E5C061E082E292E00E948E10882309F437
:10260000DDC0F89441E050E06FE770E082E292E0D4
:102610000E94E3157894D2C080E092E00E947A0E86
:10262000882309F4CBC0F89444E050E06EE670E0F3
:1026300080E092E00E94E3157894C0C063E088E6F1
:1026400092E00E948E10882351F0F89441E050E00F
:1026500065E870E088E692E00E94E31578940E94B5
:10266000B40AACC08FE792E00E947A0E80917F029C
:1026700090918002A0918102B091820220E030E02E
:1026800040E85FE3BC01CD010E941819882364F47F
:1026900080E090E0A0E8BFE380937F029093800207
:1026A000A0938102B0938202F89444E050E066E681
:1026B00070E08FE792E00E94E31578947FC08DE888
:1026C00092E00E947A0E882309F478C0F89444E0DE
:1026D00050E066E770E08DE892E00E94E3157894A0
:1026E0006DC08AE692E00E947A0E882309F466C0E3
:1026F000F89444E050E062E770E08AE692E00E94DD
:10270000E31578945BC061E089EC91E00E948E1043
:10271000882309F453C0F8940E94B40A41E050E0C1
:1027200063E870E089EC91E00E94E315789446C07C
:1027300061E08CE892E00E948E10882309F43EC08C
:10274000F89441E050E062E870E08CE892E00E948A
:10275000E315789433C061E08DE392E00E948E101F
:10276000882351F0F89441E050E064E870E08DE394
:1027700092E00E94E315789480913D02882319F03D
:102780000E9439081BC00E944B0818C01F9287E79F
:1027900090E09F938F930E94D5090F900F900F9018
:1027A0008091200283FD04C08091200280FFF8CF39
:1027B0008091200280FF02C00E945B04809142024F
:1027C00081508093420281E080930A0207C0809189
:1027D000FE01823019F481E0809327021F91089551
:1027E0000F931F93CF93DF93EC018881813209F01F
:1027F000CBC0949904C080918C028111949A85E099
:1028000080939202898199278636910509F467C0E1
:10281000873691050CF58435910509F44CC0853552
:1028200091054CF48434910509F4A4C080359105D8
:1028300009F445C0A9C08336910509F469C08436FE
:1028400091052CF48236910509F453C09DC084365D
:10285000910509F488C098C08F36910509F443C0EA
:10286000803791053CF489369105E1F08D3691056C
:1028700091F08AC08537910509F459C086379105D2
:102880002CF48237910509F47BC07EC0873791050F
:1028900009F473C079C0CE0102960E94921580930C
:1028A000CA0172C0CE0102960E9492158093430223
:1028B0000E94B40A69C064E08BE092E017C08A818C
:1028C00099278133910519F0C29729F05DC064E022
:1028D0008DE892E00BC064E08AE692E007C064E015
:1028E00080E092E003C064E08FE792E00E94BE09BE
:1028F0004BC08A8199278033910519F0C19721F047
:1029000043C010928C0240C081E080938C023CC096
:102910008A8199278033910519F0C19721F034C03D
:102920001092220231C081E0809322022DC08A8160
:1029300099278133910579F0823391051CF4C09772
:1029400039F022C08233910541F0C39741F01CC099
:102950001092680219C081E003C082E001C083E0E8
:102960008093680211C0CE0102960E949215809356
:1029700079020AC00E945B0407C00E94E80304C0F9
:10298000F8940E94960A789488818F3309F0C5C024
:10299000898199278636910509F477C08736910594
:1029A0004CF58435910509F46CC0853591058CF49E
:1029B0008C34910509F45DC08D3491052CF4833479
:1029C000910509F442C0A9C08035910509F441C0C0
:1029D000A4C08336910509F474C0843691052CF4A3
:1029E0008236910509F473C098C08436910509F4C4
:1029F00077C093C08F36910509F44BC0803791059D
:102A00008CF48936910509F468C08A3691052CF456
:102A10008836910509F469C080C08D36910509F4A6
:102A200059C07BC08337910509F445C084379105AF
:102A300024F48237910589F170C084379105E9F05B
:102A40008537910509F440C068C064E088E292E0EF
:102A500035C08A8199278133910519F0C29729F0F1
:102A60005CC064E08DE892E029C064E08AE692E010
:102A700025C064E08CEC91E021C064E083E892E042
:102A80001DC064E08BE092E019C064E080E092E059
:102A900015C064E08FE792E011C08A8199278133E5
:102AA000910519F0C29721F038C082B380781AC01E
:102AB00082B3807417C064E08FE692E00E94A70999
:102AC0002CC0809122020EC0809168020BC08091C0
:102AD0008C0208C08091CA0105C08091430202C0E7
:102AE000809179020E94CC0818C009EA11E08CE0BC
:102AF000E1ECF0E0D80101900D928A95E1F76BE0EE
:102B0000C8010E94A70923E044E062E578EB8EE16A
:102B100090E40E9446180E940809DF91CF911F910E
:102B20000F910895FC0188279927E8942191222389
:102B3000F1F02032D9F32930C9F32A30B9F32C301F
:102B4000A9F32D3099F3263789F32B3219F02D3262
:102B500021F468942191222351F0203344F02A3348
:102B600034F420530E945416820F911DF3CF811527
:102B7000910521F01EF48095909501960895E199B4
:102B8000FECF9FBB8EBBE09A99278DB30895411568
:102B9000510569F0DC01E199FECF7FBB6EBBE09A85
:102BA0006F5F7F4F0DB20D9241505040B1F70895C5
:102BB000E199FECF9FBB8EBB6DBB0FB6F894E29A36
:102BC000E19A0FBE08954115510589F0DC018FB7D8
:102BD000E199FECF7FBB6EBB0D900DBAF894E29ADF
:102BE000E19A8FBF6F5F7F4F4150504089F7089542
:102BF000E62FF72F2E2F3F2FE8944230CCF04532AE
:102C0000BCF44A3029F497FB1EF4909581959F4FB0
:102C1000642F77270E946C1B805D8A330CF0895DDE
:102C20008193862F972F009799F716F45DE25193C1
:102C3000932F822F10820C947516F52FE42FCF93CB
:102C4000FF93EF93223054F1253244F5C22FE894DC
:102C5000CA3049F497FB3EF4909580957095619544
:102C60007F4F8F4F9F4F2C2F332744275527FF939C
:102C7000EF930E94801BEF91FF91605D6A330CF02F
:102C8000695D6193622F732F842F952F6050704080
:102C90008040904041F716F4CDE2C19310828F91AD
:102CA0009F91CF910C9475167AE0979F902D879FF6
:102CB000802D910D11240895FB01DC010D90002061
:102CC000E9F7119701900D920020E1F70895FB01BB
:102CD000DC0101900D920020E1F70895FB01DC0179
:102CE00005900D920020E1F70895DC01FC010190B0
:102CF0000020E9F73297AE17BF0730F47C9160816E
:102D0000708331976D93F7CF08953F924F925F9202
:102D10006F927F928F929F92AF92BF92CF92DF92EB
:102D2000EF92FF920F931F93CF938C012B017A01A7
:102D300033246115710519F0FB0180839183E1143F
:102D4000F10449F0C7010297839728F020E030E0B2
:102D500040E050E0F7C0F801C1918F018C2F992716
:102D60000E943B1B892BB9F7CD3209F44FC0CB32FF
:102D700009F44EC0E114F10441F1F0E1EF16F10461
:102D800021F1E114F10431F4C03309F4D0C04AE078
:102D9000E42EF12C88E0E816F104F1F1E9E0EE16FA
:102DA000F1042CF5F2E0EF16F10409F4A3C0970149
:102DB000442737FD4095542F60E070E080E090E8B4
:102DC0000E94801B59016A012CC0C033D1F6F80162
:102DD0008081883711F08835A1F6F801C1810E5F36
:102DE0001F4F60E1E62EF12CF2E03F2AD3CF8AE0BC
:102DF000E816F10409F475C0E0E1EE16F104B9F645
:102E0000A12CB12CC12C28E0D22E0BC071E0372EA2
:102E1000F801C1918F01AECFA12CB12CC12C90E152
:102E2000D92E20E030E040E050E060E03701882417
:102E300077FC8094982C8C2F80538A30A8F4C82F6C
:102E4000AC2FBB27AE15BF05CCF467FD06C0A2169C
:102E5000B306C406D50658F56FEFF801C1918F018E
:102E60008C2F80538A3058F37C2F71547A3198F527
:102E7000C753AC2FBB27AE15BF053CF3411451041B
:102E800041F0662309F449C001501040F20100836B
:102E90001183832D992767FD4EC080FF31C0509567
:102EA0004095309521953F4F4F4F5F4F4BC0C40128
:102EB000B3010E944D1B9B01AC012C0F311D411D24
:102EC000511D2130F0E03F07F0E04F07F0E85F07C9
:102ED00018F661E0C2CF9C2F91569A3178F6C7550B
:102EE000AFCF3CECA32E3CECB32E3CECC32E3CE02D
:102EF000D32E97CFA12CB12CC12C80E4D82E91CF0A
:102F000057FF20C02FEF3FEF4FEF5FE702E210E0E7
:102F1000109395020093940215C0832D992781FF89
:102F2000BCCF02501040F20100831183B6CF58E0AD
:102F3000E52EF12C2FCF80FFE5CF20E030E040E000
:102F400050E8E4CFCA01B901CF911F910F91FF90D2
:102F5000EF90DF90CF90BF90AF909F908F907F9039
:102F60006F905F904F903F9008955058192EA2D1C6
:102F700001D085C1BA176207730784079507B1F1BD
:102F800088F40EF410940B2EBA2FA02D062E622F6B
:102F9000202D072E732F302D082E842F402D092E23
:102FA000952F502DFF275523B9F0591B49F0573E57
:102FB00098F0469537952795A795F0405395C9F712
:102FC00076F0BA0F621F731F841F30F487957795D0
:102FD0006795B795F040939517FA0F2E0895BF1B8C
:102FE000BB27BA0B620B730B840BF6CFDEF67FC1E7
:102FF000592F482F372F262F9FE380E87727662702
:1030000059D101D03CC1552359F0992369F09F57FC
:103010005F57951B33F442F4903811F4915805C072
:1030200046C191589F3F09F462C1BB271124621722
:103030007307840730F4660F771F881FBB1F9150FA
:1030400098F311D00F920FD00F920DD0A0E8261751
:10305000370748071B0609F0A048BA2F602D7F915B
:103060008F9100240895A0E8002462177307840755
:10307000B10528F0621B730B840BB1090A2A660F95
:10308000771F881FBB1FA69581F70895DF93CF9305
:103090001F930F93E8018C01000F111F1F3F31F4A4
:1030A0009EE481E49993899399937AC04F939923ED
:1030B0001AF40DE209939F77022F03959F938F9344
:1030C0007F936F93622F7727882799270E94F418A0
:1030D0009068AC019B0191E480E2772766270E940B
:1030E000DA195FEF4FEF0E9479192F913F914F91BD
:1030F0005F910E94B617102F013009F4002751E4A8
:1031000040E233272227621773078407950724F0CC
:103110000E9400181395F3CF9F938F937F936F9323
:103120000E94D718562F505D59930E94F4182F9182
:103130003F914F915F910E94B517905851E440E242
:10314000332722270E948C19101711F45EE259933D
:103150001A9511F718825F91EF91FF91FF93EF930A
:10316000452F442312F440954395CE01BF01861BA1
:10317000970B142F181B90E284179CF455236AF0C8
:1031800021963196E40FF11D83955A9152938A95B9
:10319000E1F792931A95E9F704C099931A95E9F724
:1031A00018828F919F918C01CF91DF91089597FBA9
:1031B0008DD09F3738F0FEE9F91B982F872F762F97
:1031C0006B2F05C091C09695879577956795F150BF
:1031D000D0F73EF490958095709561957F4F8F4F15
:1031E0009F4F0895E89403C097FB0EF4F3DFB62FCA
:1031F000672F782F892F9EE9002441C097FB66D066
:103200009F3760F40EF070C09FEB80E87727662749
:103210000895869577956795B11D93959639C8F36E
:103220002EF4BB2319F06F5F7F4F8F4FBB2727C052
:103230000ED05EF004C00BD026F001C008D019F00B
:1032400020F48FEF089580E0089581E0089597FBC2
:10325000092E052600F8689430D0E89407FC07C0D2
:10326000621773078407950721F008F40094079408
:10327000989408959A95BB0F661F771F881F112495
:103280009923A1F08823B2F79F3F59F0BB0F48F470
:1032900021F4002011F460FF04C06F5F7F4F8F4F57
:1032A0009F4F881F9795879597F908951DC09FEFA9
:1032B00080EC0895052E092607FA440F551F5F3F3D
:1032C00079F0AA27A51708F051E04795880F991FB4
:1032D0009F3F31F0BB27B91708F091E0879508951B
:1032E0009F919F911124E3CF6627772788279927FD
:1032F000089597FBEBDF992329F05F3F29F05523D1
:1033000019F00AF4F1CFD3CF940F151E01F4B7CF03
:10331000592F482F372F262FCDDF01D0B0CF99233B
:1033200039F0552329F09F575F57950F13F4CAF1D1
:10333000DECF91589F3FE1F3A62F00241124BB2735
:1033400066275527F8E0A69520F4020E131EB41F39
:10335000651F220F331F441F551FFA95A1F7F8E090
:10336000E72F7727F8E0E69520F4130EB41F651FCA
:103370007A1F330F441F551FAA1FFA95A1F7F82F84
:103380008827F69520F4B40F651F7A1F8E1F440F0F
:10339000551FAA1FEE1FFF23A1F788231AF4939548
:1033A00039F485CF000C111CBB1F661F771F881FC7
:1033B00001280895552371F1992362F059F15F9323
:1033C0004F933F932F93BBD02F913F914F915F919C
:1033D000A3DF25C09F938F937F936F935F934F934A
:1033E0003F932F93952F842F732F622FE0DEBDDD47
:1033F00091158105710561052F913F914F915F9165
:103400006F917F918F919F9121F09F775058E2DFCC
:1034100050584DCF9FE380E8772766270895092EFF
:1034200099234AF052E441EB32E76831730784078D
:10343000950758F03CCF9F7752E44EEA3CEA60355E
:1034400073078407950708F04FCF0F925FE348EBAF
:103450003AEA2BE361DFFF92EF92DF92CF9250E0E6
:103460004CE096D0ECE8F0E01ED05F2D4E2D3D2DC7
:103470002C2DCF90DF90EF90FF90FEE94595441FF3
:10348000551FF51B5527406804C04695379527956D
:103490005795FA95D2F7452F550F550B2ADF0F9008
:1034A00007FCA6CD0895092E11DFFF92EF92DF925F
:1034B000CF92BF92AF92B02CC92ED82EE72EF62E07
:1034C000A59018D0A590AA2071F09F938F937F9319
:1034D0006F936F2D7E2D8D2D9C2D0CD02F913F91B4
:1034E0004F915F9190DDAF90BF90CF90DF90EF90C4
:1034F000FF90C5CE7ED047FB406804C02F2D3E2DE7
:103500004D2D5C2DEF93FF930ADFFF91EF9171D06A
:10351000AA2707F80B24102C042607FA4068FF930B
:1035200029DDFF91992341F0882332F09A95BB0F52
:10353000661F771F881FF8CFAA9401F7089597FD9B
:10354000B6CEC4DE992309F4B2CEFF92EF92DF9299
:10355000CF92C92E9FE38F77EAEAF0E0A4DF0C2C2C
:10356000C92ED82EE72EF62E602D6E57770B872F9B
:10357000972F3ADE5FE341E332E728E1CDDE5C2DB1
:103580004D2D3E2D2F2DCF90DF90EF90FF90EECC64
:1035900097FB9CDECF93DF93D52FC42F552744276D
:1035A000332722279923D9F09F37C8F0F92F67DEF8
:1035B000592F482F372F262FF63968F4F8DD14DEFF
:1035C000C030CD0721F069937993899399939058EE
:1035D000DF91CF91CBCC9927882777276627C030FA
:1035E000CD0721F02993399349935993DF91CF91D6
:1035F00046CE559145913591259108952F923F9250
:103600004F925F926F927F928F929F92AF92BF92F2
:10361000CF92DF92EF92FF920F931F93CF93DF939E
:10362000CDB7DEB7CA1BDB0B0FB6F894DEBF0FBEFB
:10363000CDBF09942A88398848885F846E847D8448
:103640008C849B84AA84B984C884DF80EE80FD804A
:103650000C811B81AA81B981CE0FD11D0FB6F894C0
:10366000DEBF0FBECDBFED010895EE0FFF1F059029
:10367000F491E02D0994992369F4803269F08A303D
:1036800059F08C3049F08D3039F0893029F08B3089
:1036900009F40895992788270895629FD001739FA0
:1036A000F001829FE00DF11D649FE00DF11D929FDE
:1036B000F00D839FF00D749FF00D659FF00D99271D
:1036C000729FB00DE11DF91F639FB00DE11DF91F41
:1036D000BD01CF0111240895AA1BBB1B51E107C0F6
:1036E000AA1FBB1FA617B70710F0A61BB70B881F92
:1036F000991F5A95A9F780959095BC01CD01089521
:10370000A1E21A2EAA1BBB1BFD010DC0AA1FBB1FE5
:10371000EE1FFF1FA217B307E407F50720F0A21B57
:10372000B30BE40BF50B661F771F881F991F1A94C4
:1037300069F760957095809590959B01AC01BD01EE
:04374000CF01089518
:1037440000524553455420005253204F4E002F023F
:1037540046554C4C202000535552453F0052414E93
:1037640047450050415353004445435000494E00DF
:103774004D4F44450053544F5000434F4546005568
:103784004E49540054494D450050310050320042D6
:10379400454550005253204F4E00464143544F522A
:0E37A400004D44313030207265762E2000003A
:00000001FF
